:1000000009C016C015C014C013C012C011C010C062
:1000100019C00EC011241FBECFE9CDBF20E0A0E65D
:10002000B0E001C01D92A536B207E1F730D085C01F
:10003000E7CFEFE5F9E03197F1F700C00000019755
:10004000C1F708951F920F920FB60F9211248F934C
:100050009F93AF93BF938091600090916100A091B6
:100060006200B09163000196A11DB11D80936000F4
:1000700090936100A0936200B0936300BF91AF9131
:100080009F918F910F900FBE0F901F90189583B77F
:10009000826083BF8FB583608FBDF894A89580E49C
:1000A00081BD789417B886B1876886B98DE387BB20
:1000B00082E088BB9FEF96BF93EC9FBD83BFD3ECDC
:1000C00012E303E0FF24F394B199FECF8091640022
:1000D000DFBD81110FC0CFEFC6BF8C2F612F21D0A4
:1000E00090E00196A6DFC150B9F70FBD08BBF092B2
:1000F00064000EC0C0E0C6BF8C2F612F12D090E00C
:10010000019697DFCF5FCF3FB1F7C6BF1092640073
:1001100082E390E08EDFB19BFBCF82E390E089DF4A
:10012000D3CF991B79E004C0991F961708F0961B4E
:0E013000881F7A95C9F780950895F894FFCF3F
:00000001FF
